:0404000002047D3243
:01040B0032BE
:0104130032B6
:03041B0002078B4A
:0104230032A6
:01042B00329E
:010433003296
:01043B00328E
:010443003286
:01044B00327E
:010453003276
:01045B00326E
:030463000213542D
:01046B00325E
:0304730002075924
:030500000204767C
:0504760012059E80FE4E
:0E0503001213E0120A7EE58230E00543FF0489
:02051100800365
:0305130053FFFB98
:0405160053FFFD2270
:0E051A001208B8E582600F1206F3E582600851
:080528001208DF12072A80EA25
:0E05300012073FE582600F1209DDE5826008C8
:08053E00120747120A6D80EA62
:0B054600120A7EE5825401FAB40100A5
:0E0551009290120A7EE582035401FAB4010072
:0C055F00929143FE037A002092027A027F
:06056B002093034302018E
:050571008A82020A84E9
:0E05760090F25EE0FAA3E0FBA3E0FCA3E08AB3
:0E058400828B838CF01205F390F263E0F58217
:0A0592001206B890F262E0F5820252
:02059C0006E671
:07059E00121168120A987A9D
:0405A500767B0578E4
:0A05A90004EAF208EBF21205C31297
:0205B3000576CB
:0705B500121174120503127C
:0705BC00094412051A80F248
:0705C30075080075090075C1
:0605CA000A00750B00C2DF
:0405D00000C201C2A2
:0C05D4000243F54043F10275FB8243F83E
:0E05E000C043F44043A90853B9F7D2EAC28FD2
:0505EE00D2ABD2AF22E8
:0E05F300AA82AB83ACF0FDC3EA9417EB940030
:0E060100EC9400ED9400400D74A69A74909B4A
:07060F0074079CE49D5001FB
:0106160022C1
:0C061700781FEAF208EBF208ECF208EDA4
:0E062300F290000BE4F5F0C002C003C004C06A
:090631000512123085820C85834C
:05063A000D85F00EF536
:0A063F000FD005D004D003D00278DC
:0C0649001FEAF208EBF208ECF208EDF2F8
:0E0655009021D7E4F5F0121230AC82AD83AAEA
:0C066300F0FB7816741BF20874B7F20864
:0E066F00E4F208F28C828D838AF0EB1210CC3C
:0C067D00AA82AB83ACF0FDEA250CFAEB7E
:09068900350DFBEC350EFCED35DE
:040692000FFD7E00DA
:0E069600C374FF9A74019BE49CE49D50100E07
:0E06A400EDC313FDEC13FCEB13FBEA13FA801D
:0106B200E364
:0506B3008EFC8AFA2212
:0906B800AA827B00BA0102800F46
:0506C100BA0202800EE8
:0506C600BA0302800DE3
:0506CB00BA0410800CD0
:0406D0007B38800AE9
:0406D4007B18800609
:0406D8007B308002F1
:0206DC007B1091
:0806DE00744755FB4BF5FB22AC
:0906E600AA82BA020443FB0422BB
:0406EF0053FBFB229C
:0906F300E509C3950814F5822203
:0806FC00AA82AB837800E2FC46
:0A070400EC6022E5082431FDE43426
:0C070E00F0FE8A828B83E0FFA3AA82AB7E
:0C071A00838D828E83EFF005081C439A4B
:030726000880DB6D
:0107290022AD
:0A072A00AA82E5082431F582E434C8
:0A073400F0F583EAF00508439A0887
:01073E002298
:08073F00E50BC3950AF58222C7
:08074700E50A2431F582E434D7
:0A074F00F1F583E0FA050A8A822220
:0C075900C0E0C082C083C0D075D000E5B5
:0607650008B50902801432
:0A076B00C2EAE5092431F582E43406
:0A077500F0F583E0F5F905098003B3
:03077F00539AF793
:09078200D0D0D083D082D0E03247
:0E078B00C0E0C082C083C002C003C004C0052D
:0E079900C006C0D075D000C28FE5F8FA541823
:0407A7006002802D3F
:0A07AB00AB0A7C00AD0B7E00EBC32F
:0A07B5009DFBEC9EFC1BBBFF011C2A
:0A07BF00EB6012E50B2431F582E433
:0A07C90034F1F583E5F9F0050B802B
:0107D3001015
:0407D400D202800CC1
:0607D800EA30E402D20148
:0607DE00EA30E302D20044
:0E07E400D0D0D006D005D004D003D002D083F0
:0507F200D082D0E032CE
:0604D600751000C203C214
:0604DC00047801E4F2784F
:0904E20002E4F2780374FFF27ADF
:0404EB007C7B087896
:0604EF0004EAF208EBF242
:0C07F7007814740AF27582011210687800
:0B080300157440F275820412109A7800
:0B080E00147440F27582041210687828
:050819000374FFF22250
:0E081E0090F232E0FA53027FBA215190F23686
:0E082C00E0FAA3E0FB4A6006BA0143BB0040BD
:0A083A0090F233E0FABA2002800ABF
:05084400BA210280143E
:05084900BA222E801E02
:07084E007812745EF20874D9
:08085500F2F2900007021033DB
:07085D007810745EF20874CC
:08086400F2F2900007021012ED
:0C086C0090F234E0FAA3E07801EAF20216
:0208780010541A
:01087A00225B
:01087B00225A
:01087C002259
:0C087D007804E2F58208E2F58312047BA7
:0E08890090F25EE0FAA3E0FBA3E0FCA3E0FD2A
:0D089700BA4D1DBB011ABC0017BD00142096
:0508A4000411D2041252
:0E08A9001379AA82AB83ACF0FD90F231EAF035
:0108B700221E
:0A08B80090F265E0FABA1002800425
:0408C2007582002219
:0E08C60090DE0E7404F090DE14E0FA30E007CD
:0708D40090DE16E0F5822220
:0408DB007582002200
:0E08DF0090DE0E7404F090DE28E0FA90DE1633
:0C08ED00E0FB700890DE14E0FB54FEF00D
:0508F900D2068A8222F4
:0A08FE00AA82AB837806790AE2F3C0
:0B090800780BEAF208EBF27582041293
:0E0913000A9990DE16E0FA700890DE14E0FA01
:0309210054FEF091
:0109240022B0
:0E09250090DE0E7404F090DE11E0FA4401F052
:080933007440B51003D38001EC
:01093B00C3F8
:06093C009203751000D2C9
:0209420006228B
:07094400120B1130041B121D
:0E094B001379AA82ACF0FD90F231E0FBEAC312
:070959009BFA7446B5020091
:0509600050031211E438
:0A09650090F265E0FABA100280017A
:01096F002265
:0B09700090DE0E7404F0E510700B30F8
:0A097B00030B90DE11E0FA20E10307
:030985001209252F
:0A09880090DE0E7401F0780279038E
:08099200E2F5F0E3B5F00122EB
:0E099A0090DE11E0FA20E03A90DE2274A1F027
:0E09A8007420F0E4F0E4F090DE22F0E4F0744D
:0C09B60002F0E4F0780290DE22E2F09003
:0C09C200DE22E4F090DE11E04401F07849
:0A09CE0002E25483F27802E2FA78A4
:0409D80003F2D2064E
:0109DC0022F8
:0A09DD0090F265E0FABA10028004FF
:0409E70075820022F3
:0E09EB0090DE0E7404F090DE11E0FA30E110A0
:0809F900EA30E00475820022DF
:080A01007440C39510F5822238
:080A09007480C39510F58222F0
:040A1100AA82AB8387
:0A0A15007807E260527440C39510A8
:070A1F00FC7807E2B50400BA
:060A260050047807E2FC19
:0A0A2C00780DECF2780EEAF208EB08
:0E0A3600F2758204C002C003C004120ACED0C2
:0C0A440004D003D002EC2AFAE43BFB785B
:090A500007E2C39CF2EC2510F54D
:0A0A5900107440B510B6C002C003CF
:090A6300120925D003D00280A97C
:010A6C002267
:0B0A6D00E58290DE28F005107440B513
:050A7800100302092536
:010A7D002256
:060A7E007801E2F582227E
:0A0A8400AA827802E2547C4A78024C
:020A8E00F22252
:080A9000AA827802E24AF22278
:0E147C001201000202000020FB1F00220000EF
:04148A000102030157
:0E148E0009024300020100C0320904000001FF
:0E149C000202010005240020010424020205C2
:0E14AA00240600010524010001070581030A44
:0E14B800000109040100020A000000070504FB
:0B14C600024000000705840240000007
:0114D1000416
:0414D2000403090402
:0E14D600260350006F006C006F006C00750064
:0E14E400200043006F00720070006F00720065
:0A14F2006100740069006F006E00D5
:0C14FC000C0357006900780065006C00CC
:02150800D214FB
:02150A00D614F5
:02150C00FC14CD
:02150E00E603F2
:071510008025000000000827
:0404F500C205C20674
:010A9800223B
:0E0A9900AA82E4CA25E0CA33FB74202AFA744C
:0A0AA700DE3BFB780AE2FC780BE26C
:040AB100FD08E2FE5C
:0E0AB500EC60131C8A828B83E0FF8D828E839F
:080AC300F0A3AD82AE8380EACE
:030ACB00D206222E
:0E0ACE00AA82E4CA25E0CA33FB74202AFA7417
:0A0ADC00DE3BFB780DE2FC780EE231
:040AE600FD08E2FE27
:0E0AEA00EC60141C8D828E83E0FFA3AD82AE03
:090AF800838A828B83EFF080E910
:010B010022D1
:0C0B0200C20590DE017401F090DE0B745F
:030B0E0007F022CB
:0C0B110012121D400E53BE7F12122690DF
:070B1D00F265E4F0C20522BD
:0E0B240090F265E0FA701312122A43BE8000B0
:0C0B320000000090F2657402F0120B024B
:0E0B3E0090DE06E0FA90DE02E0FBEA30E00214
:020B4C00D205D0
:0E0B4E00EA30E21690F2657404F090F266E46C
:0C0B5C00F0C002C003120B02D003D00254
:060B6800EA30E102C205C3
:050B6E00EB20E0012274
:0C0B730090DE0EE4F090DE11E0FAD206F5
:0E0B7F00EA30E40B90DE117480F090F266E430
:010B8D00F077
:0D0B8E00EA30E20990DE11E4F090F266F02A
:070B9B00EA20E003020CC494
:0A0BA20090F266E0FBBB0102800345
:030BAC00020C4AEE
:0E0BAF0090DE16E0FB90F23AE0FCA3E0FD8B36
:0C0BBD00067F00C3EC9EED9F50028C03ED
:070BC900780AEBF2780879CD
:0C0BD0000BE2F308E209F3758200C0029A
:0C0BDC00C003120A99D003D0027808E28E
:0E0BE8002BF208E23400F27C0090F23AE0FDBD
:0E0BF600A3E0FE90F23AEDC39BF0EE9CA3F05C
:0E0C040090F23AE0FBA3E0FC4B600990DE1199
:060C12007440F0020CC466
:0E0C180090F232E054606007C00212087DD0F6
:010C260002CB
:0D0C270090DE0EE4F090F266E0FB700990A4
:080C3400DE117468F0020CC42B
:0E0C3C0090DE117448F090F266E4F0020CC4F1
:0C0C4A0090DE16E0FBBB086C780A740812
:080C5600F2780B7432F208740D
:0C0C5E00F2F2758200C002120A99D00266
:0E0C6A0090F266E4F090F232E054607009C03F
:080C780002120D2FD0028007CB
:070C8000C00212081ED002A1
:0D0C870090DE0EE4F090F266E0FB70089045
:070C9400DE117460F08029FD
:0E0C9B00BB012690F23AE0FBA3E0FC4B6008A0
:080CA90090DE117440F080138D
:0D0CB10090DE11744AF090F266E4F08006C7
:060CBE0090DE117440F00D
:0D0CC400EA20E16690F266E0FBBB025E9064
:0E0CD100F23AE0FBA3E0FCC3EB9420EC9400AD
:0B0CDF0050097A0A90F266E4F08004ED
:040CEA007A027B20EF
:070CEE00780DEBF2780879A4
:0C0CF5000EE2F308E209F3758200C00271
:0E0D0100C003120ACED003D00290DE11EAF039
:0C0D0F007808E22BF208E23400F27A00CF
:0E0D1B0090F23AE0FCA3E0FD90F23AECC39BAC
:050D2900F0ED9AA3F0BB
:010D2E0022A2
:0A0D2F0090F23CE4F090F23DF090E9
:090D3900F233E0FA740CB502007B
:030D42005001223B
:070D4500EA2A2A900D4C730D
:070D4C00020EF8020FAD02D8
:060D53000FBF020FAD020C
:060D59000FBF020E420272
:060D5F000D73020FBF023C
:060D65000E9B020E60026D
:060D6B000EBD020FBF02E5
:020D71000FB0C1
:0E0D730090F234E0FAA3E0FBFC7D00BC010529
:050D8100BD000280131B
:080D8600BC0205BD0002802043
:080D8E00BC0305BD0002803921
:030D9600020E1139
:070D99007808747CF2087475
:0C0DA00014F290F23A7412F0A3E4F00296
:020DAC000E1C1B
:040DAE00EA600122D4
:070DB2007808748EF208744A
:0C0DB90014F2901490E493FCA3E493FD6A
:0A0DC50090F23AECF0A3EDF0804D3F
:0E0DCF008A047D009014D1E493FE7F00C3ECF3
:060DDD009EED9F40012283
:0C0DE300E4CA25E0CA33FBEA2408F582CC
:0C0DEF00EB3415F583E493FAA3E493FBC6
:0C0DFB007808EAF208EBF28A828B83E0B1
:0A0E0700FA90F23AF0A3E4F0800B39
:0B0E110012087B90F266E0FA700122EC
:0E0E1C0090F238E0FAA3E0FB90F23AE0FCA37B
:0E0E2A00E0FDC3EA9CEB9D500890F23AEAF01E
:030E3800A3EBF039
:070E3B0090F2667402F02240
:0E0E420090F234E0FAA3E0FB90DE00EAF0EA62
:060E500060047A08800234
:020E56007A041C
:080E580090F265EAF00210546B
:0E0E600090F234E0FAA3E0FBBA0005BB0002FA
:020E6E008008FA
:080E7000BA0124BB002180142B
:0A0E780090F265E0FA7408B502007C
:0A0E8200501490F2657408F0800C23
:0B0E8C0090F2657410F01207F780016F
:010E97002238
:030E9800021054F1
:0C0E9B0090F265E0FABA10047A018002BF
:020EA7007A00CF
:080EA90090F23CEAF0781074AD
:0A0EB1003CF20874F2F29000010216
:020EBB00101213
:080EBD0090F265E0FABA1000A2
:030EC500500122B7
:0B0EC80090F236E0FAA3E0FB7C8E7D88
:0C0ED300148C828D83A3A3A3A3E493FCE2
:0A0EDF007D00C3EA9CEB9D40012258
:070EE9007810743CF208745C
:080EF000F2F290000102101261
:0E0EF80090F232E0541FFA7B00BA0005BB00F6
:030F060002801452
:080F0900BA0105BB0002802BB8
:090F1100BA0206BB0003020F82C4
:030F1A00020FAC17
:090F1D0012122350047A01800233
:020F26007A004F
:080F280090F23CEAF07810742D
:0A0F30003CF20874F2F29000020295
:020F3A00101293
:080F3C0090F265E0FABA100022
:0E0F4400500C90F236E0FAA3E0FB4A60012266
:0B0F520090F236E0FAA3E0FB7C8E7DFD
:0C0F5D00148C828D83A3A3A3A3E493FC57
:0A0F69007D00C3EA9CEB9D400122CD
:070F73007810743CF20874D1
:080F7A00F2F2900002021012D5
:0E0F820090F234E0FAA3E0FBEA540F60028024
:010F9000015F
:010F9100223D
:080F920090F265E0FABA1000CC
:030F9A00500122E1
:070F9D007810743CF20874A7
:080FA400F2F2900002021012AB
:010FAC002222
:030FAD00021054DB
:070FB0007810743CF2087494
:080FB700F2F290000212101288
:010FBF00220F
:030FC000A2052265
:0C0FC300AA8CA2BD9207C2BD438C105343
:020FCF008CFE96
:0E0FD100758900C2C5D2BDABBE74FC5B440185
:0E0FDF00F5BE000000E5BE54036007D290434B
:040FED008701C29026
:090FF100C2BDE58930E702C2052A
:0C0FFA00300509C002121223D00250CBB7
:0C100600E5BE30E6FB8A8CA20792BD22FA
:0E101200AA82AB8390F2667402F090F23AEA82
:0C102000F0A3EBF07810E2FA08E2FB7895
:07102C0008EAF208EBF222D2
:0E103300AA82AB8390F2667401F090F23AEA62
:0C104100F0A3EBF07812E2FA08E2FB7872
:07104D0008EAF208EBF222B1
:0E10540090F2667401F090F23AE4F0A3F022FC
:0610620090F266E4F022AA
:0C106800E58290DE0EF07814E2FA7B00C6
:0E10740074072AFAE43BFBC423CAC423541FAA
:0C1082006ACA541FCA6ACA30E40244E083
:0C108E0090DE10EAF090DE127401F022F7
:0C109A00E58290DE0EF07815E2FA7B0093
:0E10A60074072AFAE43BFBC423CAC423541F78
:0C10B4006ACA541FCA6ACA30E40244E051
:0C10C00090DE13EAF090DE157401F022BF
:0115170000D3
:0115180000D2
:0C10CC00AA82AB83ACF0FD781AEAF208AF
:0E10D800EBF208ECF208EDF27E007F007A00E9
:0410E6007B007C20EF
:0710EA00781DE23392087843
:0C10F1001AE225E0F208E233F208E233D4
:0E10FD00F208E233F2EE2EFEEF33FFEA33FA92
:09110B00EB33FB3008034306013D
:0C1114007816C3E2F5F0EE95F008E2F565
:0E112000F0EF95F008E2F5F0EA95F008E2F540
:0C112E00F0EB95F040227816D3E29EF41E
:0E113A00B3FEB308E29FF4B3FFB308E29AF4E9
:0C114800B3FAB308E29BF4FB781AE2440F
:0211540001F2A6
:0C115600DC92781AE2F58208E2F58308CA
:06116200E2F5F008E222B4
:0604AC00E478FFF6D8FD24
:08048A007909E94400601B7AC6
:05049200019015107837
:030497005E7593FC
:0A049A00F2E493F2A308B800020593
:0804A40093D9F4DAF27593FF1D
:0504F900781E7480F282
:071168001211891211771228
:05116F00139A0213D9E0
:0311740002120B59
:0311770053BEFB69
:0E117A00E5BE30E6FB75C68043BE0475C700B7
:011188002244
:0A11890075FF0075A00675F79922A6
:0C119300121379AA82AB83ACF0FD781E29
:0A119F00D3E29AF4FA7419B50200C5
:0C11A9005038E5FFA2E4920A400943FF21
:0711B5001075820212147490
:0E11BC0053F7EF53FFEF758201121474A2A4D3
:0A11CA00920943F710300A0343FFB7
:0111D400100A
:0C11D500121379AA82AB83ACF0FD781EE7
:0211E100EAF230
:0111E30022E9
:0E11E400C2AF75D69F75820A12147475FF0093
:0E11F20075FE0075FD0075F50075F40075F3CF
:0B120000009000641213A502000622FB
:0E120B00E5FF20E20C75820A12147430A20373
:031219000211E4DB
:01121C0022AF
:06121D00121193A2092248
:03122300A2A32261
:0412260053FFFE2252
:06122A00D2A043FF0122E7
:0C123000AA82AB83ACF0FD7823EAF20840
:0C123C00EBF208ECF208EDF27823E2FA85
:0B1248007821E2FB8AF0A4FCADF078F6
:0A12530029ECF208EDF2781FE2FC2E
:0C125D008AF0A4FDAEF07827EDF208EE58
:0A126900F2782AE2FD7826E2FE8EFC
:0A127300F0ECA42D782AF2782AE2AC
:07127D00F5117825E2FE786F
:0812840020E2F5128EF0A42512
:05128C0011782AF27840
:0712910029E2F51308E2F564
:0A129800148EF0ECA4ADF02513FE57
:0A12A200ED3514FD7829EEF208ED99
:0912AC00F27829E2F51308E2F5DD
:0812B500147824E2FF8FF0E53C
:0912BD0012A4AEF02513FDEE357C
:0A12C60014FE7829EDF208EEF28F15
:0A12D000F0EBA47826F27824E2FB8C
:0C12DA008BF0ECA4FCADF07824ECF208E2
:0A12E600EDF27822E28AF0A47822EB
:0B12F000F27820E28AF0A4FAACF0785B
:0A12FB0020EAF208ECF2781FE4F29A
:0A1305007823E4F27827E2FA08E208
:0C130F00FB08E2FC08E2FD7823E22AFA69
:0D131B0008E23BFB08E23CFC08E23DFD78E7
:0C13280027EAF208EBF208ECF208EDF204
:0A1334007827E208E208E208E278F8
:0C133E001FE22AFA08E23BFB08E23CFC3C
:0A134A0008E23D8A828B838CF022BA
:0C135400C0E0C000C0D075D000782BE2D3
:0E1360002401F208E23400F208E23400F20840
:0B136E00E23400F2D0D0D000D0E0321A
:0C137900A2BCE433FAC2BC782BE2FB08F3
:0E138500E2FC08E2FD08E2FEEA24FF92BC8BC7
:07139300828C838DF0EE2235
:0B139A0075EDBBD2BC75EBFAD2AF22A0
:0413A500AA82AB83EA
:0913A9008A048B051ABAFF011B2E
:0E13B200EC4D60227582FAC002C00312147462
:0E13C0007582FA1214747582FA121474758212
:0A13CE00F9121474D003D00280D18C
:0113D80022F2
:0804B2007831E84400600A798A
:0304BA0000759337
:0604BD00F0E4F309D8FC95
:0804C300782DE84402600C7979
:0B04CB000390F000E4F0A3D8FCD9FA85
:0713D90075D23E75D3F2222C
:02047B00E47328
:0204FE00C20B2F
:0513E00010060280155B
:0A13E50090DE0CE0FA782FF2200BE6
:0A13EF000AD20B90DE0CE0FA783011
:0113F900F201
:0C13FA00120FC0400790F265E0FA70048A
:0414060053FFEF227F
:0C140A00BA103D300B3690DE0CE0FA7B8F
:0C141600007830E2FC7D00EAC39CFAEB99
:0B1422009DFBEA30E60543FF1080034D
:03142D0053FFEF7B
:0C14300090DE0CE0FA782FD3E29AF4FA78
:05143C007460B5020020
:05144100501DC20B224A
:0414460043FF10222E
:0E144A00121379AB83ACF0FDEB035401FA6092
:051458000443FF102217
:03145D0053FFEF4B
:011460002269
:03047D0075812165
:0A048000121461E5826003020476A5
:04146100758200226E
:0B1465000000000002147000000000F6
:041470000000000078
:08147400E5826003D582EA2243
:00000001FF
